:100000000C94B6010C94EE010C94EE010C94EE01EC
:100010000C94EE010C94EE010C94EE010C94EE01A4
:100020000C94EE010C94EE010C942C1B0C94FE1B12
:100030000C9429160C94EE010C94EE010C94EE0134
:100040000C94EE010C94EE010C94EE010C94EE0174
:100050000C94EE010C94B1160C94EE010C94EE018C
:100060000C94EE010C94EE010C94EE010C94EE0154
:100070000C94EE010C94EE010C94EE010C94EE0144
:100080000C94EE010C94EE010C94EE010C94EE0134
:100090000C94EE010C94EE010C94EE010C94EE0124
:1000A0000C94EE010C94EE010C94EE018D048D0481
:1000B000B904B90421054C064C064C063F05D80589
:1000C000E905E9056B1C921C8A1D921C8A1DDE1C29
:1000D000011D8A1D581D671D3A003B0029001E00A6
:1000E0001F002000210022002300240025002600FC
:1000F00027002D002E002A004A003C003D002B0066
:1001000014001A000800150017001C0018000C004D
:10011000120013002F00300031004B003E003F0062
:10012000390004001600070009000A000B000D004A
:100130000E000F003300340028002A004E0040005B
:100140004100E10000001D001B0006001900050031
:1001500011001000360037003800E50052004D0055
:1001600042004300E000E300E20000000000000065
:100170002C0000000000000001510151500051000E
:100180004F000100010035003A003B003C003D00FB
:100190003E003F0040004100420043004400450053
:1001A0004C000100010001000100010001000100FC
:1001B0000100010001000100460047004800010065
:1001C000010001000100010001000100AA00A900D6
:1001D000A800B000010001000100010001004A0078
:1001E0000100010001000100010001000100000008
:1001F00001000100010001000100010001000100F7
:1002000001000100010001000100010001000100E6
:1002100001000100000000000000010000000000DB
:100220000000010001000100010001002803770027
:1002300069006C00620061002E00740065006300BC
:100240006800200057005400360035002D0058008B
:100250005400580000001603770069006C0062002B
:1002600061002E0074006500630068000000040354
:10027000090409023B00020100A0FA090400000180
:10028000030101000921110100012240000705813D
:100290000308000109040100010300000009211105
:1002A000010001226D0007058203200001120100F8
:1002B000020000000882651E000100010200010525
:1002C000010980A101850319012AB700150126B78C
:1002D00000950175108100C0050C0901A10185047C
:1002E00019012AA002150126A002950175108100AE
:1002F000C005010906A1018506050719E029E715D2
:100300000025019508750181020507190029EF15DF
:1003100000250195F075018102050819012905954F
:100320000575019102950175039101C0050109064A
:10033000A101050719E029E71500250195087501B8
:1003400081029501750881010507190029FF150033
:1003500026FF0095067508810005081901290595F5
:100360000575019102950175039101C011241FBE0D
:10037000CFEFDAE0DEBFCDBF04B603FE18C0809138
:10038000D5029091D602A091D702B091D8028730C1
:10039000904BA740B04B59F41092D5021092D60260
:1003A0001092D7021092D802E0E0F8E3099511E02C
:1003B000A0E0B1E0EAE2FCE302C005900D92AA38A9
:1003C000B107D9F722E0AAE8B1E001C01D92A53D2E
:1003D000B207E1F70E9487120C94131E0C940000E0
:1003E00081E0089581E008950C94F20108950C9441
:1003F000F6011F93CF93DF9300D000D01F92CDB7AB
:10040000DEB749835A836B8330918D0189819A814C
:10041000311114C0662359F0222349F00E94850847
:10042000182F682F89819A810E942E0803C00E948C
:100430005908182F69817A81812F04C00E9485088C
:1004400069817A810F900F900F900F900F90DF913C
:10045000CF911F910C94D10FFC01262F4081518127
:100460006281738184810C94F90181E00895CF93B6
:10047000DF93EC0160E00E942C02BE01DF91CF917E
:100480000C94F7010C941A110C94161108950E9403
:10049000D8060E9446022FEF84E39CE02150804062
:1004A0009040E1F700C000000C94D7160F931F9303
:1004B000CF93DF938C0161E00E942C02EC01B80124
:1004C0000E94F4018823F1F1B801CE010E9480144A
:1004D0008823C1F1B801CE010E949412882391F1C2
:1004E000B801CE010E94DC13882361F1F8018281FA
:1004F000882309F1CB358DE5D807C1F050F4C1153B
:10050000FCE5DF0781F0CF3DDC45A9F40E94BC0D7E
:1005100019C0CC35EDE5DE0761F0CD35DD4559F488
:100520000E94FF0C08C00E9447020CC00E94080DE8
:1005300002C00E940B0DC801DF91CF911F910F9156
:100540000C94F00180E0DF91CF911F910F910895FD
:100550000E9409160C94C1020E94C4020C940F164A
:1005600008950C94B00281E008950C94B3020895AC
:10057000CF93C82F0E94B1028C2F0E94B502CF9159
:10058000089580E00C94B8020E94DC140C94B80228
:100590000E94DC1490918C01891721F080938C01CA
:1005A0000C94B8020895CF93DF93CDB7DEB72B97A5
:1005B0000FB6F894DEBF0FBECDBF4F835887698753
:1005C0007A878B8761110E944B0C9E012F5F3F4FF2
:1005D00086E0F90111928A95E9F785E0FE013796E8
:1005E000D90101900D928A95E1F789819A814C8118
:1005F0005D81452B31F09F3F31F491E08F3F19F43D
:1006000003C091E001C090E090FF09C049815A8188
:100610006B817C818D819E810E946C0B05C0C9011C
:100620000E9435028111F2CF2B960FB6F894DEBFEF
:100630000FBECDBFDF91CF910895FC0180819181E4
:100640000E94C7080895CF93882309F49CC0C82F3F
:100650008238C1F40E94DC1481FD95C069E3809169
:100660000201909103010E94C4150E946D0C2FEFAE
:1006700081EE94E0215080409040E1F700C00000FE
:1006800069E319C0833801F50E94DC1480FD7BC04A
:1006900063E580910201909103010E94C4150E94BC
:1006A0006D0C2FEF81EE94E0215080409040E1F7F7
:1006B00000C0000063E580910201909103010E9457
:1006C000CF15CF910C946D0C8438C1F40E94DC14CA
:1006D00082FD59C067E480910201909103010E945C
:1006E000C4150E946D0C2FEF81EE94E021508040E4
:1006F0009040E1F700C0000067E4DDCF8CEF8C0F85
:10070000813AD0F46C2F80910201909103010E94F4
:100710004415882349F06C2F8091020190910301C8
:100720000E94CF150E946D0C6C2F80910201909158
:1007300003010E94C415C5CF80E28C0F883048F4B5
:10074000C77081E001C0880FCA95EAF70E942E0C9D
:10075000B8CFEBE5EC0FE33040F4F0E0E15CFE4FA6
:10076000808190E0CF910C940215C85AC73158F49B
:10077000EC2FF0E0EE0FFF1FEF5EFE4F80819181C6
:10078000CF910C941815CF910895882309F45BC07C
:10079000682F823879F40E94DC1481FF54C069E329
:1007A00080910201909103010E94C4150E946D0C7A
:1007B00069E310C08338B1F40E94DC1480FF43C0A9
:1007C00063E580910201909103010E94C4150E948B
:1007D0006D0C63E580910201909103010E94CF1599
:1007E0000C946D0C843879F40E94DC1482FF2BC0C9
:1007F00067E480910201909103010E94C4150E9458
:100800006D0C67E4E7CF8CEF860F813A18F380E236
:10081000860F883048F4677081E001C0880F6A95C0
:10082000EAF70E94340CDCCF8BE5860F833020F48E
:1008300080E090E00C940215685A673120F480E063
:1008400090E00C94181508951F93CF93DF93182F01
:10085000EB010E942303209741F08FE99FE001976D
:10086000F1F700C000002197F6CF812FDF91CF91E3
:100870001F910C94C503893319F060E070E002C049
:1008800060E570E00C942404882321F00E942E0C73
:100890000C946D0C0895882321F00E94340C0C9464
:1008A0006D0C0895CF92DF92EF92FF920F931F93FA
:1008B000CF93DF937C01D62FC72FFC0112810581D6
:1008C00002950F700E94240C8823B9F01123A9F01F
:1008D0008C2F807F803421F080E28D0F883068F08B
:1008E00080919B0282FD09C082E00E94CD0C0E9493
:1008F000240C91E0D82ED92601C0D12CCC2EC29444
:100900008FE0C8228C2D90E08C30910508F0C4C196
:10091000FC01EA5AFF4F0C94BE1D8C2F807FCF70D4
:10092000882311F0C295C07F112399F0CC2309F4DC
:100930009FC180E28D0F883010F0D11104C08C2F40
:100940000E942E0C03C08C2F0E943E0C0E946D0C46
:100950008FC18D2F0E94C503CC2309F49DC180E275
:100960008D0F883038F1DD2329F18C2F0E94440C43
:1009700024C08C2F807FCF70803211F0C295C07F51
:10098000DD2319F0D130A1F13DC080919B0282FF9F
:1009900017C0112349F0CC2329F08C2F0E942E0C74
:1009A0000E946D0C80E065C180E00E94C503CC23ED
:1009B00009F472C18C2F0E94340C0E946D0C6CC122
:1009C000112371F0002341F0013031F40E944E0CEC
:1009D0008C2B0E94560C60C10E944E0C8C2B1DC0AB
:1009E000002319F0013009F457C10E94630C25C09F
:1009F000112321F0063008F04FC10EC0053008F079
:100A00004BC11BC0112361F0002331F0F701858138
:100A100080FF2EC18F7085838C2F0E9444043CC1BF
:100A2000002359F0D93309F034C1FFEF07EE13E08A
:100A3000F15000401040E1F72AC18C2F0E944B0476
:100A40002BC18C2F86958695837019F0813061F0CB
:100A500023C1112321F08D2F9C2F937002C080E0C1
:100A600090E00E94021520C1112321F08D2F9C2FB0
:100A7000937002C080E090E00E94181515C18C2F81
:100A8000837009F047C011110BC12D2F22952695B7
:100A90002770220F220F6D2F6F70862F90E0A0E03D
:100AA000B0E0022E04C0880F991FAA1FBB1F0A9432
:100AB000D2F7D4FF10C04FE050E060E070E004C017
:100AC000440F551F661F771F2A95D2F74095509502
:100AD0006095709503C040E050E0BA01C695C69598
:100AE000C3708A019B01082B192B2A2B3B2BC901B0
:100AF000B801C23049F058F4C13019F00E944407DF
:100B0000CFC00E943207CCC00E945607C9C00E94C5
:100B10003007C6C0112319F08C2F817001C0869553
:100B2000882309F4BDC02D2F229526952770220F0A
:100B3000220F6D2F6F70862F90E0A0E0B0E0022EA4
:100B400004C0880F991FAA1FBB1F0A94D2F7D4FFB5
:100B500010C04FE050E060E070E004C0440F551F4B
:100B6000661F771F2A95D2F740955095609570952E
:100B700003C040E050E0BA01C695C695C3708A0133
:100B80009B01082B192B2A2B3B2BC901B801C23022
:100B900049F058F4C13019F00E94090881C00E9440
:100BA000F7077EC00E941B087BC00E946A0778C0BE
:100BB000CF70112339F08C2F0E9490078D2F0E9447
:100BC00044046EC08D2F0E944B048C2F0E94B107ED
:100BD00067C0D23F21F128F4D03F41F0D13FC1F0AE
:100BE00043C0D33F19F1D43F79F03EC0112341F007
:100BF000053008F051C08C2F8F710E94D6074CC071
:100C0000063008F049C0F7CF80919B0282FF18C0E0
:100C1000112339F08C2F8F710E9490073DC0112352
:100C2000C9F38C2F8F710E94B10736C0112329F0B0
:100C30008C2F8F710E947B072FC00E9476072CC0DB
:100C4000112349F0CF718C2F0E94900763E08C2F05
:100C50000E94B20C21C081E00E94CD0C0230E0F075
:100C600082E00E94CD0C18C0112331F0002391F2D4
:100C70008D2F0E94230310C0002399F2D93349F429
:100C80001FEF27EE33E0115020403040E1F700C065
:100C900000008D2F0E94C50388EF8C0D843020F456
:100CA0000E94DC140E94B802DD20C9F00E94200CD2
:100CB00080FD15C0F70112820E941A0C0E94900755
:100CC000C7010E9490060E941A0CDF91CF911F91DC
:100CD0000F91FF90EF90DF90CF900C94B107DF91D0
:100CE000CF911F910F91FF90EF90DF90CF900895DB
:100CF0000F931F93CF93DF93EC01688179818A81F1
:100D00000E94D2088C010E942D080E941E07B80183
:100D1000CE010E945204DF91CF911F910F9108954F
:100D2000CF93DF93EC01988189812B813C81232B28
:100D300031F08F3F31F481E09F3F19F403C081E02F
:100D400001C080E080FD1DC0CE010E9456028111CD
:100D500010C00E94240C8823A1F08A81882389F086
:100D600080919B0282FD0DC082E0DF91CF910C94B7
:100D7000CD0CCE010E947806CE01DF91CF910C946C
:100D80003702DF91CF91089580E090E00E94021534
:100D900080E090E00E9418150E944B0C0C946D0CA2
:100DA00080910201909103010E94DA150C94C4060F
:100DB0000E943B0C0C94D00692959F70963079F06F
:100DC00010F4925001C09A50923068F4803F69F05C
:100DD00018F4883E40F409C0843F29F406C0883ED8
:100DE00020F0813F11F080E0089581E00895FC013A
:100DF000808191810E94C7080E94DC060895CF93EC
:100E0000DF9300D000D01F92CDB7DEB70F900F90C8
:100E10000F900F900F90DF91CF910895CF93DF93B4
:100E200000D000D000D0CDB7DEB726960FB6F8942C
:100E3000DEBF0FBECDBFDF91CF9108950895089515
:100E40000C941F070C9420070E9422076093C9018D
:100E50007093CA018093CB019093CC010C94C4068B
:100E60000C9424070F931F930091C9011091CA019C
:100E70002091CB013091CC01602B712B822B932BD5
:100E80001F910F910C9424070F931F930091C90198
:100E90001091CA012091CB013091CC0160237123C4
:100EA000822393231F910F910C9424070F931F9378
:100EB0000091C9011091CA012091CB013091CC0160
:100EC00060277127822793271F910F910C94240785
:100ED0000C941F070E9468076093C5017093C601B8
:100EE0008093C7019093C8010C94C40660E070E041
:100EF000CB010C946A070F931F9341E050E060E030
:100F000070E08A019B0104C0000F111F221F331FD4
:100F10008A95D2F7C901B8011F910F910C946A0705
:100F20000F931F9341E050E060E070E004C0440F75
:100F3000551F661F771F8A95D2F78091C501909142
:100F4000C601A091C701B091C8018A019B01082B7D
:100F5000192B2A2B3B2BC901B8011F910F910C941F
:100F60006A070F931F9341E050E060E070E004C017
:100F7000440F551F661F771F8A95D2F740955095ED
:100F8000609570958091C5019091C601A091C701AF
:100F9000B091C8018A019B01082319232A233B230E
:100FA000C901B8011F910F910C946A070F931F9309
:100FB00041E050E060E070E004C0440F551F661F40
:100FC000771F8A95D2F78091C5019091C601A091B3
:100FD000C701B091C8018A019B01082719272A2758
:100FE0003B27C901B8011F910F910C946A070F9319
:100FF0001F930091C5011091C6012091C701309146
:10100000C801602B712B822B932B1F910F910C9495
:101010006A070F931F930091C5011091C60120919B
:10102000C7013091C80160237123822393231F914C
:101030000F910C946A070F931F930091C5011091B3
:10104000C6012091C7013091C8016027712782270E
:1010500093271F910F910C946A07089521E1929FA5
:10106000800D1124E82FE695E695E695877051E00E
:1010700001C0550F8A95EAF785E0E89FF001112439
:10108000E257FE4F20E030E070E04081CB01022EBD
:1010900002C0969587950A94E2F78170819584271E
:1010A0008523842781932F5F3F4F2530310569F7D2
:1010B000089521E1929F800D1124682F6695669511
:1010C0006695982F977085E0689FB001112440E0E5
:1010D00050E080E0FB01E40FF51FE257FE4F208156
:1010E00030E0092E02C0369527950A94E2F7217068
:1010F0003327042E01C0220F0A94EAF7822B4F5F98
:101100005F4F4530510531F70895BF92CF92DF927E
:10111000EF92FF920F931F93CF93DF938C01C090B8
:10112000C501D090C601E090C701F090C801809140
:10113000C9019091CA01A091CB01B091CC01C82AFC
:10114000D92AEA2AFB2ACFE1D0E0D701C6010C2E2A
:1011500004C0B695A795979587950A94D2F780FD18
:1011600004C0219790F7B12C07C0BC2EB8018C2F7A
:101170000E94E40F0197A9F38B2DDF91CF911F916E
:101180000F91FF90EF90DF90CF90BF900895CF9395
:10119000DF93EC010E948508BE010E94E40FDF91FD
:1011A000CF9108951F93CF93DF93EB0190918D0121
:1011B000992321F0CB010E94C70813C0882349F06E
:1011C000CB010E948508182F682FCE010E942E089F
:1011D00004C0CB010E945908182FBE01812F0E9424
:1011E000E40FDF91CF911F9108951F93CF93DF9369
:1011F000C091CD0116E08091CE01C81799F0D0E0E2
:101200001C9FF0011D9FF00D1124E153FE4F408102
:10121000518162817381848195810E940E0721969C
:10122000C770E9CFDF91CF911F9108954091FF01E1
:1012300050910002609101027091020280910302BC
:10124000909104020C940E07EF92FF920F931F935C
:10125000CF93DF938091040282958F7009F065C06F
:1012600080910102882309F460C08091CD01F09043
:10127000CE011091FF010091000260910202709175
:10128000030291E01F3F09F090E0C0910001D0916E
:101290000101292F96E0E92E8F1509F446C061154A
:1012A000710521F00F3F21F030E003C031E001C0B3
:1012B000322F90E030FD36C0E89EF001E99EF00D3F
:1012C0001124DF01A153BE4F11963C9111973013A9
:1012D00029C03C91311326C012963C9112973111CE
:1012E00021C013964D915C911497461B570B4C17D8
:1012F0005D07C0F4809104028F70806180930402C6
:10130000EC52FE4F80818F70806180838FEF91E07F
:101310000E949006DF91CF911F910F91FF90EF9067
:101320000C94F50801968770B7CFDF91CF911F918C
:101330000F91FF90EF9008959F92AF92BF92CF923E
:10134000DF92EF92FF920F931F93CF93DF93CDB76E
:10135000DEB761970FB6F894DEBF0FBECDBF8C012C
:1013600085E0F801DE011D9601900D928A95E1F766
:10137000D8011296EC909091FF01E091000220912B
:101380000202309103022115310531F0EF3F31F4B3
:1013900081E09F3F19F403C081E001C080E0B82FD5
:1013A000B1709B2E80FD47C1D8014C9111965C9184
:1013B00011971396AD90BC9014978FEFC82E81E0D3
:1013C000D82EF0900102B501621B730B2091000131
:1013D00030910101FF2009F4D9C080910402621705
:1013E000730708F095C0282F207F09F052C05E13C4
:1013F00013C0491311C0FE2CE1100EC08F70806124
:10140000809304020E941609C6010E9490068091F2
:101410000402F80185834DC1AB2831F05F3F31F400
:1014200081E04F3F19F403C081E001C080E080FDFE
:1014300003C081E08E2502C080E090E0F82FF170BB
:10144000FF2E80FF1CC08091CD012091CE0136E09F
:10145000821709F40BC190E0389FF001399FF00D1D
:101460001124E153FE4F6181561306C0608146137B
:1014700003C06281E61203C001968770E9CFFE2C9B
:10148000EE2009F416C18091040281608093040269
:1014900054C05E1306C0491304C0E11002C0F80135
:1014A00099C0C8010E94F706882361F1EE2051F12E
:1014B00020910402822F82958F7090E0029774F041
:1014C0008091FF019091000298878F831986BB86D7
:1014D000AA862C87CE0107960E94900686E0F80126
:1014E000AFEFB1E001900D928A95E1F70E942409D7
:1014F0000E9416090AC05E1711F1C8010E94F70682
:1015000081112CC0C8010E949006FF24F394D1C021
:10151000282F207F81F77A2DB98AA88A6E2D898994
:101520000E94FF068FEF91E00E94900686E0D601B0
:101530001D928A95E9F70E941609F12CBAC0491349
:10154000DCCFE110DACFF8018583C8010E94900654
:1015500086E0D6011D928A95E9F7ABC0EE2091F2A4
:1015600020910402822F82958F7090E002970CF4F4
:10157000B5CF8091FF01909100029A8389831B82ED
:10158000BD82AC822E83CE010196A6CF621773076F
:1015900008F044C0FE2CEE2009F4B4CF5E1330C036
:1015A00049132EC02091040220FD21C0822F829574
:1015B0008F70482F50E041155105C9F0F80125837F
:1015C0004F30510541F08F5F982F9295907F822F79
:1015D0008F70892B8583C8010E94900686E0F801F0
:1015E000AFEFB1E001900D928A95E1F73CC086E043
:1015F000F801AFEFB1E001900D928A95E1F759C083
:10160000C8010E94F706811169CF809104028160B0
:1016100080930402C8010E9490064BC07A2DB98ABB
:10162000A88A6E2D89890E94FF0686E0D6011D9248
:101630008A95E9F718C0EE2009F464CFC8010E942A
:10164000F706F82E882309F45DCF86E0F801AFEFA6
:10165000B1E001900D928A95E1F78FEF91E00E9441
:101660001D030E9424090E94160923C04D875E872E
:101670008D859E850E94C708292F22952F702230C4
:1016800028F49F7039F0811105C00BC0243028F474
:101690009F7049F4805E883020F0C8010E94900657
:1016A0009F2CF92C06C0D80115969C91907F91F73C
:1016B000F8CF8F2D61960FB6F894DEBF0FBECDBF69
:1016C000DF91CF911F910F91FF90EF90DF90CF901E
:1016D000BF90AF909F9008951F93CF93DF93CDB7A6
:1016E000DEB72C970FB6F894DEBF0FBECDBF4F8389
:1016F000588769877A878B879C87CE0107960E94D7
:101700009C098823D1F09F8188852A853B85232BDE
:1017100031F08F3F31F481E09F3F19F403C081E045
:1017200001C080E080FD47C04F81588569857A857A
:101730008B859C850E940E073EC086E0FE01379691
:10174000DE01119601900D928A95E1F7FF81E885FF
:101750006A857B856115710531F0EF3F31F481E0D9
:10176000FF3F19F403C081E001C080E080FD23C089
:101770002091CE0130E0C9010196877099274091F0
:10178000CD0150E084179507F1F1F983EA837D8359
:101790006C8396E0929FD001939FB00D1124A153CA
:1017A000BE4FFE01319601900D929A95E1F780931C
:1017B000CE010E94F50816E08091CD019091CE01F6
:1017C000891771F1189FC001112481539E4F0E9407
:1017D0009C09882329F1E091CD011E9FF00111247D
:1017E000E153FE4F408151816281738184819581F3
:1017F0000E940E078091CD0190E001968770992795
:101800008093CD01D9CF0E94D8061092CE011092BC
:10181000CD01EFEFF1E086E0DF011D928A95E9F757
:101820002C960FB6F894DEBF0FBECDBFDF91CF91DF
:101830001F91089580912502859585958595089538
:10184000809125028770089590912502977081E01C
:1018500009F480E00895809148020895909148022B
:10186000892B80934802089580959091480289239E
:10187000809348020895109248020895909147027B
:10188000892B809347020895809590914702892380
:10189000809347020895109247020895809126028E
:1018A000089508950C94510C0C94520C90919B0245
:1018B00092FD08C090912602981721F0809326028D
:1018C0000C94540C089580912602882329F01092DC
:1018D000260280E00C94540C0895CF93DF93E0919E
:1018E0000201F0910301809148028083E09102019E
:1018F000F0910301908180914702892B8083809130
:101900002602882381F0E0910201F0910301908189
:10191000892B808380910201909103010E942E15F2
:1019200081110E94630CC0910201D091030140E239
:1019300050E065E072E0CE010E94C41D892B69F081
:1019400080E2FE01A5E0B2E001900D928A95E1F7F8
:10195000CE01DF91CF910C94E814DF91CF910895DF
:101960000C94510C90919B0292FD10C098E0899FBD
:1019700090011124262B209325020E94900780912C
:1019800025028595859585950C94B00C0C9490074F
:101990001092250280E00C94B00C209125028095D5
:1019A000822380932502982F977099F430E0482F76
:1019B000082E000C550B2417350759F090919B0207
:1019C00092FD07C08595859585950E94B1070C9479
:1019D000C80C089590919B0292FB222720F92817AA
:1019E00069F080FB92F990939B0280919A0290910A
:1019F0009B020E94380D82E00C94CD0C08958091DA
:101A00009B0282FB882780F991E089270C94EA0CDD
:101A100081E00C94EA0C80E00C94EA0C6FEF7FEF0D
:101A200080E090E00C94FD1D80E090E00E94D91DC4
:101A300021E0893E9E4F09F020E0822F089582E048
:101A400090E00C94D11D83E090E00C94D11DCF93D5
:101A500084E090E00E94D11DC82F82E290E00E94B5
:101A6000D11D2C2F30E0A901582BCA01CF91089528
:101A7000CF93C92F682F84E090E00E94DF1D6C2F68
:101A800082E290E0CF910C94DF1DAB01BC018FE0AE
:101A900090E00C94F11DAB01BC0183E190E00C944B
:101AA000F11D60E070E0CB010C944B0D60E070E044
:101AB000CB010E94450D0C94510D69EE7EEF80E044
:101AC00090E00E94FD1D60E082E090E00E94DF1D3A
:101AD00060E083E090E00E94DF1D1092C901109247
:101AE000CA011092CB011092CC0160E084E090E03A
:101AF0000E94DF1D60E082E290E00E94DF1D60E056
:101B000085E090E00E94DF1D60E086E090E00E94AA
:101B1000DF1D6FEF87E090E00E94DF1D40E050E0A6
:101B2000BA0188E090E00E94F11D60E08DE090E055
:101B30000E94DF1D40E050E0BA0188E190E00E9481
:101B4000F11D60E087E190E00E94DF1D40E050E081
:101B5000BA018CE190E00E94F11D60E070E080E24B
:101B600090E00E94FD1D40E050E0BA0188E190E065
:101B70000E94F11D0C94560D0C945D0D682F8EE0A3
:101B800090E00C94DF1D0E949616609361027093A2
:101B90006202809363029093640260935D0270938B
:101BA0005E0280935F0290936002089585B780681B
:101BB00085BF85B7806885BF089581E008950C943E
:101BC000DD0D08950C94E10D0C94E10D0C94E40DE1
:101BD0000C94E10D0C94E80D0C94E10D0E94D60DCF
:101BE00080EC90E10E94D2140E94EC0D0C94EA0D5E
:101BF0000E94E20D0C94E10D0E94DA100C94B702E1
:101C00000E9481160E94DE110E94FC0D0C94E60DCC
:101C10002F923F924F925F926F927F928F929F92FC
:101C2000AF92BF92CF92DF92EF92FF920F931F93EA
:101C3000CF93DF93CDB7DEB72D970FB6F894DEBF05
:101C40000FBECDBF0E94F311282E81110E94C30D3B
:101C500089E492E09D878C8700E010E0302E802F91
:101C60000E94FE102B013C01EC85FD858191919134
:101C7000A191B191FD87EC875301420188269926F5
:101C8000AA26BB2681149104A104B104B1F40F5F0C
:101C90001F4F0530110511F78FEF89838A831B824F
:101CA0000E948A168160782F9D838C8349815A8196
:101CB0006B818D810E94D30251C08091650281FDAC
:101CC0000E940A111B86C12CD12C7601C394D50128
:101CD000C4018C219D21AE21BF21892B8A2B8B2B06
:101CE00091F10E94DF0D8823D1F0FB85FE833F82B6
:101CF0004C205D206E207F2081E045284628472823
:101D000009F480E088870E948A168160782F9A877C
:101D100089874E815F8168858A850E94D302000F82
:101D2000111F000F111FF801E75BFD4F80819181AA
:101D3000A281B381C826D926EA26FB26C082D18299
:101D4000E282F3820BC08B858F5F8B87CC0CDD1C0E
:101D5000EE1CFF1C813109F0BACF99CF81E0211030
:101D600001C080E02D960FB6F894DEBF0FBECDBF48
:101D7000DF91CF911F910F91FF90EF90DF90CF9067
:101D8000BF90AF909F908F907F906F905F904F909B
:101D90003F902F9008950E94080E0C94C802CF9394
:101DA000DF930E94E90FEC01811522E59207E8F527
:101DB000811531E5930708F0B6C0883E910528F5F6
:101DC000803E910508F0E9C0883A910570F4853AA3
:101DD000910508F07AC08130910509F473C008F4C8
:101DE000D9C0049708F0D9C0D5C08F3B910508F041
:101DF000D1C0C85AD0E0CC0FDD1FCE5BDE4F0990BA
:101E0000D881C02DCE019464C9C0811540E59407E6
:101E100008F069C0811550E4950708F060C09A95F4
:101E200081159F4108F4B9C0B5C0811536E5930707
:101E300028F5811545E5940708F092C0811554E511
:101E4000950708F087C0AC0143705527282F2695C9
:101E50002695C115D34508F06CC081E090E002C022
:101E6000880F991F4A95E2F740E2249F90011124C0
:101E7000EC01C22BD32BCE019C6890C081152AE5C2
:101E8000920780F4811539E5930708F072C0811537
:101E900048E5940708F47EC0D82FCC27CE01806F88
:101EA000906A7CC090568115904208F073C08D2FC7
:101EB0008F710E947D10DD27D0628F71AE01582B8B
:101EC000CA016CC081E090E069C0C55AD0E0C05939
:101ED000DE4F8881C82FD0E0CE0190645FC0DF70F4
:101EE000CE01906A5BC074E0969587957A95E1F78C
:101EF000282F23703C2F337081E090E002C0880FC0
:101F0000991F3A95E2F79C68AC01522B9A019C2FDD
:101F10009F709695969550E2959FE0011124C90116
:101F20008C2B9D2B3BC0D82FCC27CE01816F906A84
:101F300035C081E090E002C0880F991F4A95E2F712
:101F400050E2259F90011124EC01C22BD32BCE012E
:101F50009A6824C0D82FCC27CE01846F906A1EC007
:101F60000E947D108F7190E0D82FCC27CE01906217
:101F700015C08F700E947D1094E0D695C7959A95F4
:101F8000E1F7CF70D0E0DC2FCC27D0699E01282B61
:101F9000C90104C080E090E001C0CE01DF91CF9183
:101FA000089525E5829FC0011124FC0121E1729F63
:101FB000E00DF11D1124E60FF11DEE0FFF1FE85299
:101FC000FF4F8591949108950E94D10F0E94CF0EEA
:101FD00008958238910569F1B0F48133910509F4CF
:101FE0006DC048F48932910509F463C08A329105C5
:101FF00009F469C008958533910509F455C0893302
:102000009105B9F00895833E910569F138F4803E59
:102010009105B1F0823E910509F10895863E910542
:10202000A9F1873E9105B9F1843E910509F064C09C
:1020300023C020919A0220FD4FC021FD4DC008957C
:1020400080919A0280FD44C080919B0280FF44C031
:1020500080919A0284FD42C083EE4DC080919A0225
:1020600082FF38C0F5CF80919A0282FD33C0809103
:102070009B0280FD31C0ECCF80919B0281FF32C07A
:1020800080919A0284FD2AC087EE35C080919A0221
:1020900083FF26C0F5CF80919A0283FD21C08091F5
:1020A0009B0281FD1FC0ECCF80919A0285FD1CC070
:1020B0001DC080919A0285FD19C016C080919A02B8
:1020C00086FD16C017C080919A0286FD13C010C00D
:1020D00089E311C082EE0FC080EE0DC080E00BC01E
:1020E00086EE09C084EE07C089E205C085E303C01F
:1020F0008AE201C081E390E0089590919A0292FFF4
:102100000DC0282F2871283019F4877F846006C0FD
:10211000282F2471243011F48B7F886093FF0DC029
:10212000282F2871283119F4877E846106C0282F52
:102130002471243111F48B7E886120919B0220FF51
:102140000DC0382F3871383019F4877F816006C090
:10215000382F3171313011F48E7F886021FF0DC02E
:10216000282F2871283119F4877E816106C0282F15
:102170002171213111F48E7E886194FD877E08954E
:1021800080E008950C940E0D0E94F3118FE39CE9FA
:102190000197F1F700C000000E94F31180E00E9457
:1021A000FE1060FF04C00E94C2100C94D716089560
:1021B0000C94C4100E94140D811102C00E94BC0D29
:1021C0000E941F0D809365020E94270D90939B0231
:1021D00080939A020E94D8100E94230D682F70E00D
:1021E00080E090E00E9430076091C5017091C601C7
:1021F0008091C7019091C8010C94680724E0829FE8
:10220000C0011124FC01E055FD4F60817181828184
:1022100093810895089580EA8A95F1F7089500C0A2
:1022200008950C940B1108950C9413110C9414112F
:102230000C9413110C941811F894E82FE295EF7098
:10224000F0E031A1282F2F7081E090E001C0880FCD
:102250002A95EAF7982F9095932391A392A1892B21
:1022600082A3789408950F931F93CF93DF93C4E8CC
:10227000D1E089918F3F11F00E941C1181E0C93893
:10228000D807B9F7C3E7D1E004E811E089918F3F9F
:1022900011F00E941C110C171D07C1F7DF91CF919F
:1022A0001F910F9108954F925F926F927F928F923C
:1022B0009F92AF92BF92DF92EF92FF920F931F9384
:1022C000CF93DF938C01C62FD0E0CE018C579E4F69
:1022D0007C01FC0190819F3F09F460C0D62EF894E8
:1022E000E92FE295EF70F0E081A19F7021E030E0EE
:1022F00001C0220F9A95EAF7822B81A382A1209533
:10230000282322A378940E940F11E3E7F1E024E848
:1023100031E0412C512C32014394812C912C5401F9
:1023200081918F3F99F0A82FA295AF70B0E0909661
:102330004C9150E08F70BA0102C0759567958A95EF
:10234000E2F760FD03C0D301C20103C080E090E06A
:10235000DC01882A992AAA2ABB2A440C551C661C2F
:10236000771C2E173F07E1F6F70180818F3F11F0B0
:102370000E941C1161E081149104A104B10409F4CC
:1023800060E08D2D0E941111CC0FDD1FCC0FDD1FE1
:10239000C00FD11F88829982AA82BB82DF91CF9120
:1023A0001F910F91FF90EF90DF90BF90AF909F90A3
:1023B0008F907F906F905F904F9008950E9433119F
:1023C00084E1E0EBF2E0DF01982F1D929A95E9F7A6
:1023D000ECE9F2E0DF011D928A95E9F785E00E94C1
:1023E0003E120C944202FF920F931F93CF93DF9300
:1023F000CDB7DEB764970FB6F894DEBF0FBECDBF82
:102400008E010F5F1F4F84E1F80111928A95E9F761
:10241000F12C6F2DC8010E945311F394F5E0FF12C7
:10242000F8CF44E150E0B8018CE992E00E94C41D6D
:10243000FF24F394009709F4F12C892B41F084E1F7
:10244000F801ACE9B2E001900D928A95E1F72F2DE9
:1024500045E060EB72E08CE992E00E943F120E943E
:1024600044028F2D64960FB6F894DEBF0FBECDBF29
:10247000DF91CF911F910F91FF9008950895FF92E2
:102480000F931F93CF93DF93F82ED92F8B01C42F77
:10249000222349F081E0809368020E948A1690937B
:1024A000670280936602809168028823F1F0809130
:1024B0006602909167020E94A2160597B0F0EF2D78
:1024C000FD2FD80180E090E04C2F50E08417950755
:1024D00054F401911191219131910D931D932D93FC
:1024E0003D930196F3CF10926802DF91CF911F9137
:1024F0000F91FF9008950E9484180E94000E0C9482
:1025000090180E9494180E94CB0E0C94AE180E9452
:1025100028160E946B180E94EE0D0E947B120E94EA
:1025200081120E94F80DFBCFCF93DF93EC01FB01EA
:102530008281882309F43CC1C430FDE5DF0760F4E3
:10254000CB3F9CE5D90788F49E0122503C452431BD
:10255000310508F02EC109C0C236EDE5DE0729F0CD
:10256000C63AFDE5DF0709F024C10E94270D9093CC
:102570009B0280939A02C1318CE5D80709F4C6C04A
:1025800008F042C0C930ECE5DE0709F49BC000F555
:10259000C5308CE5D80709F485C078F4C330ECE584
:1025A000DE0709F478C008F07AC0C230DC4509F0D3
:1025B000F5C080919A028160EFC0C7309CE5D907D1
:1025C00009F478C008F07AC080919A028061E4C072
:1025D000CD30FCE5DF0709F487C058F4CB309CE52B
:1025E000D90709F479C008F07BC080919A0288600D
:1025F0006FC0CF30FCE5DF0709F480C008F082C06F
:1026000080919A02877FC8C0CE3F9CE5D90709F424
:1026100071C000F5C531FCE5DF0709F485C068F439
:10262000C3319CE5D90709F475C008F095C00E9434
:10263000D80680919A028F77AFC0CC3FFCE5DF07C8
:10264000A9F108F054C0CB3FDC4509F0A7C0809148
:102650009B0240C0C230EDE5DE0709F489C058F4A2
:10266000C1158DE5D80709F45AC008F069C08091FA
:102670009B0282602FC0C236EDE5DE0709F47CC004
:10268000C63AFDE5DF0709F481C0C330DD4509F036
:1026900085C080E06EC080919A0282607DC080918A
:1026A0009A0216C080919A02886076C080919B023F
:1026B00082604FC080919A0280626EC080919A02BF
:1026C00080646AC00E94D80680919A02806864C0C3
:1026D000846062C081603DC080919A028E7F5CC040
:1026E00080919A028D7F58C080919A0216C0809185
:1026F0009B0218C080919B028D7F2BC080919A0213
:102700008F7E4AC080919A028F7D46C080919A0246
:102710008F7B42C080919A02877F8B7F3DC08091E2
:102720009B028D7F8E7F15C080919A0282FB2227AB
:1027300020F991E0922790FB82F990FB83F92CC05D
:1027400080919B02982F909591708E7F892B90FBA2
:1027500081F980939B0222C00E94D80680919A0240
:1027600087FB222720F991E0922790FB87F914C07C
:1027700081E00E94BE0D12C080919A0284FB222744
:1027800020F991E0922790FB84F906C080919A028B
:10279000982F909590FB80F980939A0280919A02ED
:1027A00090919B020E94380D0E94D80680E001C0E3
:1027B00081E0DF91CF910895CF93DF9386319C45DF
:1027C00041F5EB010E942B0C982F8A812091020188
:1027D00030910301882379F09A7A81E009F480E04E
:1027E00080936902911102C069E201C065E3C901E9
:1027F0000E94C4150AC080916902811102C069E279
:1028000001C065E3C9010E94CF150E946D0C80E0F4
:1028100001C081E0DF91CF9108950F931F93CF9373
:10282000DF93C42FD22FFC0182818823C9F040930B
:102830006C020E948A1690936B0280936A0280E277
:102840008C0F883008F057C0C77081E001C0880F36
:10285000CA95EAF7DF91CF911F910F910C94440430
:1028600080916C02481330C080916A0290916B0293
:102870000E94A216883C910538F510E21D0FCD1775
:10288000B9F080E28C0F883040F4C77081E001C05D
:10289000880FCA95EAF70E944B04183028F581E0AA
:1028A0009D2F977001C0880F9A95EAF70E94440403
:1028B000802F0E943B041830F0F4D77081E001C0F3
:1028C000880FDA95EAF70AC080E28C0F883098F416
:1028D000C77081E001C0880FCA95EAF7DF91CF91F8
:1028E0001F910F910C944B04802FDF91CF911F917A
:1028F0000F910C943B04DF91CF911F910F9108959C
:102900000F939C01CB01243F4CE5340731F188F44F
:10291000293DFCE53F07D9F02A3D4CE5340779F124
:10292000283D3C45A9F506E221EE41EE68ED7CE547
:102930002BC0263FFCE53F07E1F0A8F0273F3C45D0
:1029400039F507E225EE46EE67EF7CE51DC007E2AC
:1029500025EE45EE69ED7CE517C006E221EE40EE7E
:1029600064EF7CE511C007E225EE44EE65EF7CE5FF
:102970000BC006E221EE42EE66EF7CE505C008E200
:1029800021E045EE6AED7CE50E940D1480E008C070
:10299000FC018281882319F010926C0201C081E051
:1029A0000F91089590938B0180938A0108959093DD
:1029B0007202809371020895E0917102F0917202A7
:1029C000309721F00190F081E02D099480E0089586
:1029D000E0917102F0917202309799F0209110010C
:1029E000222359F020919A0227FF07C0DC012C9185
:1029F00011962C93119726E02C930280F381E02D01
:102A00000994089520916F023091700228173907B8
:102A100071F09093700280936F02E0917102F091D7
:102A20007202309721F00680F781E02D0994089515
:102A300020916D0230916E022817390771F0909342
:102A40006E0280936D02E0917102F09172023097F4
:102A500021F00084F185E02D09940895FC0132965F
:102A600080911001882331F080919A0287FF02C083
:102A70009EE101C096E080E0915028F02191222350
:102A8000D9F38F5FF9CF0895662351F1209110019A
:102A90002223E9F020919A0227FF19C0462F46957C
:102AA000469546954E31E0F4677021E030E002C073
:102AB000220F331F6A95E2F7FC01E40FF11D8281BA
:102AC00090E02823392381E0232B69F409C0FC011D
:102AD000329608962191621729F0E817F907D1F785
:102AE00080E0089581E008959C01FC0132969FEFFB
:102AF00080E04191461789F09F3F19F4411101C0D0
:102B0000982F8F5F8630A9F79F3F39F0F901E90FC1
:102B1000F11D97FDFA956283089508959C012A5F3F
:102B20003F4FFC014281461301C012820196821779
:102B30009307B9F70895262F2695269526952E31C9
:102B400068F4FC01E20FF11D677021E030E001C084
:102B5000220F6A95EAF78281282B22830895262F77
:102B60002695269526952E3170F4FC01E20FF11D75
:102B7000677021E030E001C0220F6A95EAF72095E6
:102B8000828128232283089520911001222329F095
:102B900020919A0227FD0C949B150C94741520919A
:102BA0001001222329F020919A0227FD0C94AF15E1
:102BB0000C948E1520911001FC013296222331F0E5
:102BC00080919A0287FF02C08EE101C086E0DF019A
:102BD0001D928A95E9F7089508950C94EC1583E009
:102BE000809373020C94ED15811102C081E001C045
:102BF00082E0809373020C94ED150C94F41581E03F
:102C0000809373020C94ED150C94FF1508950C94A9
:102C100006160C9407160C9406160C9406160C94C3
:102C20000616CF930E940D160E94F3110E940B16F8
:102C3000C0E08C2F0E94FE10672B682B692B29F4B3
:102C4000CF5FC530B1F780E001C081E0CF9108953A
:102C500008951F920F920FB60F9211248F939F9396
:102C6000AF93BF9380917402811113C08091C4020D
:102C70009091C502A091C602B091C7024196A11DD4
:102C8000B11D8093C4029093C502A093C602B09375
:102C9000C702BF91AF919F918F910F900FBE0F9080
:102CA0001F9018958091CC02843031F10E94A802C7
:102CB0001092740220E488E190E00FB6F894A89591
:102CC000809360000FBE2093600083B7817F846093
:102CD00083BF83B7816083BF7894889583B78E7FE5
:102CE00083BF0FB6F894A8958091600088618093A7
:102CF0006000109260000FBE08950E94D8060C94E8
:102D0000AC0282E084BD93E095BD9AEF97BD8093BD
:102D10006E0008952FB7F8948091C4029091C50277
:102D2000A091C602B091C7022FBF08952FB7F894A3
:102D30006091C4027091C5028091C6029091C70251
:102D40002FBF08959C014FB7F8948091C4029091D1
:102D5000C502A091C602B091C7024FBF821B930B60
:102D6000089578941F920F920FB60F9211248F93AB
:102D70009F93AF93BF938091C4029091C502A0919D
:102D8000C602B091C7020196A11DB11D8093C40275
:102D90009093C502A093C602B093C702BF91AF91B2
:102DA0009F918F910F900FBE0F901F90189581E00B
:102DB0008093E00080E28093D8001092C9008FE1F8
:102DC0009EE40197F1F700C0000087E090EBDC0182
:102DD0008093D5029093D602A093D702B093D802E5
:102DE0009CE088E10FB6F894A895809360000FBE30
:102DF00090936000FFCF8091980208950895CF933B
:102E0000DF9320911001222339F020919A0227FFAD
:102E100003C060E222E002C068E021E02093E90004
:102E20002FEF3091E800215035FD06C035ED3A9581
:102E3000F1F700002111F5CF2091E80025FF1DC01A
:102E4000EC0180911001811105C040E050E068E084
:102E500070E003C070E040E050E0CE010E94201915
:102E60008091E8008E778093E80080E2FE01A8E779
:102E7000B2E001900D928A95E1F7DF91CF9108952C
:102E80008093750270937702609376028091CC02F2
:102E9000843001F582E08093E9008FEF9091E800A3
:102EA000815095FD06C095ED9A95F1F700008111CE
:102EB000F5CF8091E80085FF0DC040E050E063E071
:102EC00070E085E792E00E9420198091E8008E77FB
:102ED0008093E8000895BC0184E00C944017BC0185
:102EE00083E00C94401708958091CB02811109C0B2
:102EF0000E94B11A0E940E1B8091E20084608093B0
:102F0000E20008951092CB0208950C94041660918B
:102F1000C80281E0611101C080E00C94EF1590912E
:102F2000CC0281E0943009F080E06091C8020C94FA
:102F3000F41542E061EC81E00E942A1A42E261EC61
:102F400082E00E942A1A9091CC0281E0943009F02C
:102F500080E06091C8020C94FD158091CE02833010
:102F600009F461C030F4813071F0823009F49AC004
:102F700008958A3009F486C08B3009F46CC089301A
:102F800009F0A8C020C08091CD02813A09F0A2C00A
:102F90008091E800877F8093E8008091D102909132
:102FA000D202892B21F460E288E792E003C060E05E
:102FB00080E090E070E00E946B198091E8008B77D0
:102FC0008093E80008958091CD02813209F082C09B
:102FD0008091D1029091D202029708F07BC080913B
:102FE000E800877F8093E8008091E80082FD05C0BB
:102FF0008091CC028111F8CF6DC02091F3008091B7
:10300000F20090E0922B029731F48091F100813030
:1030100011F0863021F48091F10080939802809124
:10302000E8008B7753C08091CD02813A09F052C0FD
:103030008091D1029091D202892B09F04BC08091EE
:10304000E800877F8093E8008091E80080FFFCCF54
:103050008091100136C08091CD028132D9F58091E6
:10306000D1029091D202892BA9F58091E800877F47
:103070008093E8000E945F1A8091CF028093100134
:103080000C94D8068091CD02813221F58091E80020
:10309000877F8093E8000E945F1A8091D00280931E
:1030A000990208958091CD02813AA1F48091E800BF
:1030B000877F8093E8008091E80080FFFCCF8091BB
:1030C00099028093F1008091E8008E778093E80068
:1030D0000C945F1A089584B7877F84BF0FB6F89465
:1030E000A8958091600088618093600010926000D4
:1030F0000FBE90E080E80FB6F89480936100909343
:1031000061000FBE0C94FF150E94B11A0E940E1BA5
:10311000E2EEF0E080818460808378940C94A31DBB
:1031200084E091E00C94D7148091CC028530A9F40E
:103130008091CC02853079F40E9452168091CA02A7
:103140008823B1F30E941116882391F30E940A1973
:103150000E94D806EDCF0C947D16089508950C9426
:10316000B118292F332723303105C9F060F42130FD
:10317000310581F02230310509F044C08BE390E045
:1031800022E732E043C021323105E1F0223231053D
:1031900049F138C082E190E02DEA32E037C099274A
:1031A0008130910549F028F0029761F5ECE2F2E0F8
:1031B00005C0EEE6F2E002C0E6E5F2E0849190E0C0
:1031C0009F0124C06115710541F061307105D1F492
:1031D00089E090E02DE932E019C089E090E024E830
:1031E00032E014C06115710541F06130710551F490
:1031F0008DE690E02FEB32E009C080E490E02CE215
:1032000033E004C080E090E020E030E0FA01318358
:103210002083089580E189BD82E189BD09B400FE63
:10322000FDCF8091D8008F7D8093D8008091E00001
:1032300082608093E0008091E00081FDFCCF0895E2
:10324000CF92DF92EF92FF920F931F93CF93DF9372
:10325000EC018B017A010E947E1A811133C0E114C6
:10326000F10439F0F70180819181081B190BC80F17
:10327000D91FC12CD12C0115110519F18091E8003D
:1032800085FD16C08091E8008E778093E800E114F8
:10329000F10449F0F70180819181C80ED91ED182D5
:1032A000C08285E00FC00E947E1A882321F30AC0E5
:1032B00089918093F10001501109FFEFCF1ADF0AC5
:1032C000DACF80E0DF91CF911F910F91FF90EF90C7
:1032D000DF90CF9008952091D3023091D402261729
:1032E000370748F06115710539F42091E8002E7711
:1032F0002093E80001C0B901FC0120E061157105CF
:1033000079F18091CC028823F1F18530F1F180913F
:10331000E80083FD3CC08091E80082FD2EC08091D2
:10332000E80080FFEBCF2091F3008091F20090E065
:10333000922B6115710551F08830910538F4219177
:103340002093F100615071090196F3CF21E00897B5
:1033500009F020E08091E8008E778093E800CECFDE
:103360002111CFCF0AC08091CC02882361F0853033
:1033700061F08091E80083FD0AC08091E80082FF3F
:10338000F2CF80E0089582E0089583E0089581E01F
:1033900008952091D3023091D4022617370748F0C0
:1033A0006115710539F42091E8002E772093E8002B
:1033B00001C0B901FC0120E06115710591F1809116
:1033C000CC02882309F440C0853009F43FC08091C5
:1033D000E80083FD3DC08091E80082FD2FC0809110
:1033E000E80080FFE9CF2091F3008091F20090E0A7
:1033F000922B6115710559F08830910540F42491A4
:103400002093F1003196615071090196F2CF21E0CD
:10341000089709F020E08091E8008E778093E8001B
:10342000CBCF2111CCCF0AC08091CC02882361F090
:10343000853061F08091E80083FD0AC08091E8004A
:1034400082FFF2CF80E0089582E0089583E008953E
:1034500081E00895982F973068F59093E9009817C8
:1034600039F07091EC002091ED005091F00003C014
:10347000242F762F50E021FD02C09F5FECCF3091CA
:10348000EB003E7F3093EB003091ED003D7F3093B9
:10349000ED003091EB0031603093EB007093EC0065
:1034A0002093ED005093F0002091EE0027FDE5CF32
:1034B00080E008958F708093E90081E00895809105
:1034C000CD0287FF11C08091E80082FD05C0809188
:1034D000CC028111F8CF11C08091E8008B770BC02E
:1034E0008091CC02882349F08091E80080FFF8CFDA
:1034F0008091E8008E778093E80008952091E400A1
:103500003091E50095E64091EC00842F817040FFFA
:1035100023C08091E80080FD1DC08091CC028823EB
:1035200099F0853099F08091EB0085FD11C04091B4
:10353000E4005091E5002417350729F3915011F06C
:103540009A01E1CF84E0089582E0089583E0089530
:1035500081E0089580E008954091E80042FFDDCFCA
:1035600008950E941F1B0E94271BE0EEF0E080815F
:1035700081608083E8EDF0E080818F77808319BCE3
:10358000A7EDB0E08C918E7F8C9380818F7E8083BD
:103590001092CB0208950F931F93CF93DF930E9455
:1035A0001F1B0E94271BC8EDD0E088818F7788837E
:1035B00088818068888388818F7D888319BC109278
:1035C000CC021092C8021092CA021092C90200EEF8
:1035D00010E0F80180818B7F8083888181608883FF
:1035E00042E060E080E00E942A1AE1EEF0E0808193
:1035F0008E7F8083E2EEF0E0808181608083808135
:1036000088608083F80180818E7F808388818061DB
:103610008883DF91CF911F910F910895E8EDF0E03D
:1036200080818F7E8083E7EDF0E080818160808300
:1036300084E082BF81E08093CB020C94CB1AE8ED4A
:10364000F0E080818E7F80831092E20008951092D6
:10365000DA001092E10008951F920F920FB60F92B8
:1036600011242F933F934F935F936F937F938F9387
:103670009F93AF93BF93EF93FF938091E10082FFFD
:103680000BC08091E20082FF07C08091E1008B7F38
:103690008093E1000E94A21D8091DA0080FF1FC08C
:1036A0008091D80080FF1BC08091DA008E7F8093CC
:1036B000DA008091D90080FF0DC080E189BD82E1F0
:1036C00089BD09B400FEFDCF81E08093CC020E9449
:1036D000741705C019BC1092CC020E948217809109
:1036E000E10080FF19C08091E20080FF15C0809149
:1036F000E2008E7F8093E2008091E20080618093FF
:10370000E2008091D80080628093D80019BC85E0E7
:103710008093CC020E9487178091E10084FF30C023
:103720008091E20084FF2CC080E189BD82E189BDE7
:1037300009B400FEFDCF8091D8008F7D8093D80022
:103740008091E1008F7E8093E1008091E2008F7E86
:103750008093E2008091E20081608093E20080919A
:10376000C802882311F084E007C08091E30087FD40
:1037700002C081E001C083E08093CC020E948F17D9
:103780008091E10083FF29C08091E20083FF25C082
:103790008091E100877F8093E10082E08093CC02FA
:1037A0001092C8028091E1008E7F8093E1008091A9
:1037B000E2008E7F8093E2008091E200806180933E
:1037C000E20042E060E080E00E942A1A8091F0006E
:1037D00088608093F0000E948517FF91EF91BF9160
:1037E000AF919F918F917F916F915F914F913F9199
:1037F0002F910F900FBE0F901F9018951F920F9250
:103800000FB60F9211242F933F934F935F936F93B3
:103810007F938F939F93AF93BF93CF93DF93EF9358
:10382000FF93C091E900CF708091EC00D82FD17048
:1038300080FDD0E81092E9008091F000877F8093AE
:10384000F00078940E94421C1092E9008091F000F0
:1038500088608093F000CD2BCF70C093E900FF917A
:10386000EF91DF91CF91BF91AF919F918F917F9118
:103870006F915F914F913F912F910F900FBE0F90DD
:103880001F9018951F93CF93DF93CDB7DEB7AA97FC
:103890000FB6F894DEBF0FBECDBFEDECF2E0809125
:1038A000F100819322E0E53DF207C9F70E94AD17D0
:1038B0008091E80083FF2EC18091CD029091CE02CD
:1038C000492F50E04A30510508F024C1FA01EE5961
:1038D000FF4F0C94BE1D803821F0823809F01AC1C8
:1038E00008C08091C9029091CA02992389F0826030
:1038F0000FC08091D1028F70873008F00BC1809388
:10390000E9008091EB0085FB882780F91092E9009F
:103910009091E800977F9093E8008093F1001092D7
:10392000F100D1C0282F2D7F09F0F4C0882319F0B1
:10393000823061F0EFC08091CF02813009F0EAC09F
:10394000933009F080E08093CA022EC08091CF02AC
:1039500081112AC08091D1028F702FEF280F26305D
:1039600008F0D8C08093E9002091EB0020FF1CC034
:10397000933021F48091EB00806214C09091EB00B1
:1039800090619093EB0021E030E0A90102C0440F68
:10399000551F8A95E2F74093EA001092EA00809161
:1039A000EB0088608093EB001092E9008091E800C2
:1039B000877F8093E8000E945F1AACC08111AAC083
:1039C0001091CF021F778091E3008078812B809344
:1039D000E3008091E800877F8093E8000E945F1AEF
:1039E0008091E80080FFFCCF8091E30080688093A5
:1039F000E300111102C082E001C083E08093CC0299
:103A000089C08058823008F085C08091CF029091A3
:103A1000D0028C3D53E0950779F583E08A838AE2F2
:103A200089834FB7F894DE01139620E03EE051E21F
:103A3000E32FF0E050935700E49120FF03C0E2959C
:103A4000EF703F5FEF708E2F90E0EA3010F0C79676
:103A500001C0C0968D939D932F5F243149F74FBFCE
:103A60008091E800877F8093E8006AE270E0CE01F1
:103A700001960E946B1916C06091D1027091D2021A
:103A8000AE014F5F5F4F0E94AF18BC01892B09F454
:103A900041C09091E800977F9093E80089819A81D6
:103AA0000E94C9198091E8008B778093E80032C0AA
:103AB000803881F58091E800877F8093E8008091CD
:103AC000C8028093F1008091E8008E7772CF811157
:103AD00021C08091CF029091D00299270297D4F40F
:103AE0008091E800877F8093E8008091CF028093E7
:103AF000C8020E945F1A8091C802811106C080919D
:103B0000E30087FD02C081E001C084E08093CC0225
:103B10000E9499178091E80083FF0AC08091E80015
:103B2000877F8093E8008091EB0080628093EB00B8
:103B3000AA960FB6F894DEBF0FBECDBFDF91CF912E
:103B40001F9108950895CF938091CC028823A1F00E
:103B5000C091E900CF709091EC00892F817090FDA9
:103B600080E8C82B1092E9008091E80083FD0E9454
:103B7000421CCF70C093E900CF910895EE0FFF1F54
:103B80000590F491E02D0994FB01DC0104C08D91B6
:103B90000190801921F441505040C8F7881B990BBF
:103BA0000895F999FECF92BD81BDF89A992780B505
:103BB0000895A8E1B0E042E050E00C94051E262FE5
:103BC000F999FECF92BD81BDF89A019700B4021613
:103BD00039F01FBA20BD0FB6F894FA9AF99A0FBEC1
:103BE00008950396272F0E94E01D0E94DF1D252FB8
:103BF0000E94E01D242F0C94E01D0196272F0E94A7
:103C0000E01D0C94DF1DDC01CB01FC01F999FECF16
:103C100006C0F2BDE1BDF89A319600B40D92415054
:0A3C20005040B8F70895F894FFCF64
:103C2A00C8002702FB16FF1673176F176B17FE16CD
:103C3A0001E200E900EA00B500B600B700CD008352
:103C4A0001CC008A01920194012102230224022557
:103C5A0002260227022A02B300B4006F0070008114
:103C6A008283E200E900EA00B500B600B700CD00A1
:103C7A008301CC008A0192019401210223022402C9
:103C8A002502260227022A02B300B4006F00700040
:103C9A008182833730F595313233939267663635B0
:0A3CAA0034979694F0F1F4F6F70059
:00000001FF
